:0A21E70000010202030304040505D1
:1009AE00E4F565F564F563F562C212C20FC211C2B9
:1009BE00101220B81207B67E187F008E0A8F0B75A4
:1009CE00121875131275081875091C751018751103
:1009DE005175141875157FEE54E07003020AF57503
:1009EE0066007567808E688F69C374A99FFF74183F
:1009FE009ECF2402CF3400FEE48F618E60F55FF54A
:100A0E005EF55DF55CF55BF55AAF61AE60AD5FAC62
:100A1E005EAB5DAA5CA95BA85AC3120C4E5026E5CC
:100A2E0067255DF582E566355CF58374CDF0E55D91
:100A3E002401F55DE4355CF55CE4355BF55BE4358E
:100A4E005AF55A80C4E4F55DF55CF55BF55AAF6175
:100A5E00AE60AD5FAC5EAB5DAA5CA95BA85AC3127B
:100A6E000C4E5031AE5CAF5DE5692FF582E5683E08
:100A7E00F583E0FDE5672FF582E5663EF583EDF043
:100A8E00EF2401F55DE43EF55CE4355BF55BE435A2
:100A9E005AF55A80B985660A85670B74002480FF63
:100AAE00741834FFFEC3E5139FF513E5129EF5127D
:100ABE00C3E50D9FF50DE50C9EF50CC3E50F9FF5F7
:100ACE000FE50E9EF50EC3E5099FF509E5089EF5A7
:100ADE0008C3E5119FF511E5109EF510C3E5159FAE
:100AEE00F515E5149EF514D2E843D82090E668E09B
:100AFE004409F090E65CE0443DF0D2AFD288D28A51
:100B0E00C2A8C2AA43E808D2FB90E680E020E10525
:100B1E00D213121EC190E680E054F7F0538EF8C245
:100B2E0012301005120592C2103012291216FE5004
:100B3E0024C21212203D200F1690E682E030E70408
:100B4E00E020E1EF90E682E030E604E020E0E412FF
:0A0B5E001EF01217FE12136B80C781
:1005920090E6B9E070030206431470030206C02419
:1005A200FE700302074324FB700302063D1470032E
:1005B200020637146073146076240560030207A2F2
:1005C20012222040030207AE90E6BBE024FE602226
:1005D20014603324FD601114602224067048E50A79
:1005E20090E6B3F0E50B8037E51290E6B3F0E51341
:1005F200802DE50C90E6B3F0E50D8023E50E90E644
:10060200B3F0E50F801990E6BAE0FF121F1CAA06AC
:10061200A9077B01EA494B600DEE90E6B3F0EF903B
:10062200E6B4F00207AE0207A71221510207AE128A
:10063200220C0207AE121B180207AE12213F02075C
:10064200AE12222240030207AE90E6B8E0247F6099
:100652001514601924027063A20FE43325E0FFA28F
:1006620011E4334F8041E490E740F0803F90E6BCD4
:10067200E0547EFF7E00E0D394807C0040047D0144
:1006820080027D00EC4EFEED4F24E7F58274213EA0
:10069200F583E493FF3395E0FEEF24A1FFEE34E609
:1006A2008F82F583E0540190E740F0E4A3F090E6F6
:1006B2008AF090E68B7402F00207AE0207A71222BC
:1006C2002440030207AE90E6B8E024FE601624023E
:1006D20060030207AE90E6BAE0B40105C20F02075A
:1006E200AE0207A790E6BAE0705590E6BCE0547EF1
:1006F200FF7E00E0D394807C0040047D0180027D77
:1007020000EC4EFEED4F24E7F58274213EF583E4C2
:1007120093FF3395E0FEEF24A1FFEE34E68F82F5DE
:1007220083E054FEF090E6BCE05480131313541F90
:10073200FFE0540F2F90E683F0E04420F0806D80BC
:1007420064122226506690E6B8E024FE6019240264
:10075200705A90E6BAE0B40104D20F804F90E6BA24
:10076200E064026047803E90E6BCE0547EFF7E007B
:10077200E0D394807C0040047D0180027D00EC4E39
:10078200FEED4F24E7F58274213EF583E493FF33B7
:1007920095E0FEEF24A1FFEE34E68F82F583800818
:1007A200120080500790E6A0E04401F090E6A0E03D
:0307B2004480F090
:0107B5002221
:0300330002221C8A
:04221C0053D8EF3272
:1020B800758CE0758AC0E58954F04401F589758E00
:0820C80003D28CD2A9D2AF2291
:03005B00020F97FA
:0D0F9700C0E0C083C082C0D075D000C0078C
:100FA400AF91530780EF6480600302109F53917FD9
:100FB400300D0302109DE55064017043D3E538946D
:100FC400C8E5379400500302109D902473E54FF058
:100FD400D394C8E54E9400401DD3E54F94B0E54E3C
:100FE40094045012E5389460E53794095008752C40
:100FF40001755000D20285374E85384F021097E5AF
:101004005064027061C3E53894C8E53794004048E1
:10101400D3E53894C8E53794004010D3E53894B04C
:10102400E53794045005752C008027D3E53894B037
:10103400E5379404400FD3E53894ACE537940D506C
:1010440004052C800DD3E53894ACE537940D4008A5
:10105400052C753700753800E52C652D703BF5506F
:10106400F537F5388033E550B4022ED3E5389401D2
:10107400E5379400402374722535F582E43424F571
:1010840083E538F00535052CE52CB40F06755000C2
:0B109400752C00753700753800C20D88
:0B109F00D007D0D0D082D083D0E03248
:101800001201000200000040181615A80000010295
:1018100000010A0600020000004001000902350034
:1018200001010080FA0904000005FF00000007051F
:101830000102400000070582020002000705810244
:1018400040000007058602000200070508020002AA
:101850000009022E0001010080FA0904000004FFC3
:101860000000000705010240000007058202400059
:101870000007050202000200070581024000000483
:1018800003090410035100480059002D0043004390
:10189000004400160351004800590038003100345C
:0B18A00000410020002000200000009C
:100CED00608024BF03050303020201070000000218
:100CFD00000002001332120A080C08080000000060
:100D0D000000003F0305030202020107000000007E
:100D1D00020002001312320A120C0C08000000002F
:100D2D000000003F030F030303030107000000024F
:100D3D00000002001332120A080C0808000000001F
:100D4D000000003F030C0302030201070000000036
:100D5D00020002001332120A120C0C0800000000EF
:100D6D000000003F60242546000000000000000048
:100D7D000000000000000000000000000000000066
:100D8D0000000000000000000000000047253F802B
:060D9D00000010CA4E0028
:1015BC0090E60174CAF090E6F574FFF090253FE0D8
:1015CC0090E6F3F0902540E090E6C3F0902541E0E2
:1015DC0090E6C1F0902542E090E6C2F0902544E000
:1015EC0090E6C0F0902545E090E6F4F075AF0774F6
:1015FC0024F59A74BFF59B759DE4E4F59EFF90E687
:10160C007BE090E67CF00FBF80F490E67174FFF005
:10161C00F5B490E672E04480F043B680000000E43C
:10162C0090E6C4F000000090E6C5F0902546E090EE
:10163C00E6C6F0902547E090E6C7F0902548E0908C
:10164C00E6C8F0902549E090E6C9F090254AE09074
:10165C00E6CAF090254BE090E6CBF090254CE0905C
:0B166C00E6CCF090254DE090E6CDF0BC
:011677002250
:03004300021700A1
:0300530002170091
:101700000220D00002211600022100000220E80081
:10171000021DBE00021D4A000222280002222900EA
:1017200002222A0002222B00021E900002129700C1
:1017300002222C0002222D00021D0B00021B77004A
:1017400002222E000222290002222F000222300053
:10175000022231000222320002223300022234002F
:101760000222350002222900022229000222290039
:1017700002223600022237000222380002223900FB
:1017800002223A0002223B0002223C0002223D00DB
:1017900002223E0002223F000222400002224100BB
:1017A000022242000222430002224400022245009B
:0817B00002224600022247005C
:101EF00090E682E030E004E020E60B90E682E030FD
:101F0000E119E030E71590E680E04401F07F147EAF
:0C1F1000001217B890E680E054FEF022AA
:10203D0090E682E044C0F090E681F0438701000015
:04204D00000000226D
:101EC10030130990E680E0440AF0800790E680E054
:101ED1004408F07FDC7E051217B890E65D74FFF0D0
:0F1EE10090E65FF05391EF90E680E054F7F02227
:021F1C00A90713
:101F1E00AE14AF158F828E83A3E064037017AD01EC
:101F2E0019ED7001228F828E83E07C002FFDEC3E36
:091F3E00FEAF0580DF7E007F008C
:011F47002277
:1017B8008E6F8F7090E600E054187012E570240167
:1017C800FFE4356FC313F56FEF13F570801590E6DE
:1017D80000E05418FFBF100BE57025E0F570E56FC9
:1017E80033F56FE5701570AE6F7002156F4E6005BA
:0617F80012205180EE22D8
:102051007400F58690FDA57C05A3E582458370F9A2
:01206100225C
:100DA300C1834224BD00004224B200004224B400A7
:100DB3000041241000412411004124B70002310BEB
:100DC30016C100012600C1054124B600C109C106B0
:100DD300014B00044300000000043C0000000060DD
:100DE300402472000000000000000000000000002A
:100DF30000000000000000000000000000000000F0
:100E030000000000000000000000000000000000DF
:100E130000000000000000000000000000000000CF
:100E2300000000013500015001012DFF012C0002DB
:100E3300370000024E0000014D000157000255002B
:100E4300000233C350012B19C10BC18DC102C10C68
:090E5300013B00013900013000EF
:101F48008F6A9024527403F0E4A3F07A247B527DC4
:101F5800027F4112209C9024527401F0A3E56AF09C
:0B1F68007A247B527D027F4102209C06
:0B21D100C2B6C2B48FB1D2B4D2B622A5
:0B21DC00D2B6C2B48FB1D2B4D2B6228A
:1016EB00AE05AD077F151221D1AF051221D1AF0683
:0316FB000221D1F8
:10212C00AE05AD077F751221D1AF051221D1AF06D7
:03213C000221D1AC
:041FF000AC05AB078A
:101FF4007D5FE4FF1216EB7D3FFF12212CFEE4FD12
:10200400AF031221DCAF041221DC0DBD60F20EBE61
:0220140040EC9E
:0120160022A7
:061C2B008B6A8A6B896CD4
:101C3100E4F56DF56E900001120B68FC700C7D5F90
:101C4100FF1216EB7D3FFF02212CBCFF2DD2B67592
:101C51006D00756E02C2B4AB6AAA6BA96C856E8207
:101C6100856D83120B68F5B1D2B4056EE56E700215
:0A1C7100056DB482E0E56DB401DBFF
:011C7B002246
:10143600C2B77FC87E00122069D2B77FAE1221D113
:101446007FA01221D17F721221D17FA11221D1E476
:10145600FF1221D17FA21221D1FF1221D17FA41226
:1014660021D17FA81221D17F3F1221D17FAD122138
:10147600D17F8E1221D17FB01221D17F0B1221D1C3
:101486007FB11221D17F311221D17FB31221D17FB9
:10149600F01221D17F8A1221D17F641221D17F8B54
:1014A6001221D17F781221D17F8C1221D17F641233
:1014B60021D17FBB1221D17F3A1221D17FBE1221C9
:1014C600D17F3E1221D17F871221D17F061221D1F1
:1014D6007F811221D17F911221D17F821221D17F6A
:1014E600501221D17F831221D17F7D1221D17FAF6E
:0314F6000221D1FF
:1007B60090E600E054E74410F000000000000090CE
:1007C600E61074A0F000000090E60B7401F090E6CD
:1007D6001274E0F0000000E490E613F000000090D0
:1007E600E61474E2F000000090E61574A0F0000034
:1007F6000090E6D27402F090E6047480F0000000E7
:100806007402F00000007406F00000007408F000A6
:100816000000E4F00000001215BC90E6187408F021
:1008260000000090E619F000000090E61AF00000C3
:100836000090E61BF0000000E490E671F075B47FCE
:1008460075A07F90E672F075B6FF75B1FF90E67001
:10085600F075B2FF75B5FFC28CD2B0D2B11221B716
:1008660090E61074A0F000000090E611F000000081
:1008760090E65EE04408F0000000E490E68DF000AB
:10088600000090E65EE04404F0000000E490E7C05B
:10089600F090E7C4F0A3F0A3F0A3F090E7F0F09097
:1008A600E68F7440F000000090E65EE04440F00001
:1008B60000007E027F0090F800E4F0A3DFFCDEFA81
:1008C60090E6987402F0000000E490E699F00000CB
:1008D600007E027F0090F800E4F0A3DFFCDEFA90D1
:1008E600E65EE04480F0000000E490E69CF0000044
:1008F6000090E69DF00000007F9AFE1221F1752817
:10090600007529B47551017552907531107532B85C
:1009160075530675542C12221490E67AE054FEF0B4
:10092600E4FD7F901221637F647E001217B87DFF7D
:100936007F421221637F647E001217B87D827F4E4C
:10094600122163753AFF43A020E4F54290E782E561
:100956003AF090E781E542F01221B7D20D755001C9
:10096600753327753410752B0A1219C37F887E13C9
:100976001220691219C37FB87E0B1220697F887E08
:10098600131220691221C41214367DAA7FAA121FDF
:10099600F0D2F9C2F8E4F54B90E7C0E54BF043A07E
:0709A6001053917F53A0F0F4
:0109AD002227
:0E21A900EF2401FBE43EFA7D047F4802208013
:101F9E00E542C313FFC374809F9024BEF0E4940007
:101FAE009024BDF0E542D394004006753AFF43A05D
:091FBE0020E542700353A0DF226C
:1011B200E4FC9024B9E0FEA3E02400FDEC3EFC90A8
:1011C2002410E0FEA3E07A002400FFEA3EFEC3ED15
:1011D2009FFFEC9EFE9024B2F0A3EFF09024B5E0C6
:1011E2002FF09024B4E03EF0D3EF9450EE6480945C
:1011F2008050129024B2E0FAA3E0FBC394B0EA64F8
:1012020080947F501C9024B3E025E0FE9024B2E04D
:10121200339024BDF0A3CEF0E49024B4F0A3F08088
:10122200337C007D14AF03AE02120BB7AC06AD07E0
:101232009024B4E0FEA3E07802C333CE33CED8F9D3
:101242002DFFEC3EFE7C007D0A120BC99024BDEE00
:10125200F0A3EFF0D39024BEE094FF9024BDE064AD
:101262008094804006E4F0A374FFF0C39024BDE0B4
:10127200648094805004E4F0A3F09024BDE0FEA3C7
:10128200E0FF7C007D02120BC9C3747F9FF0E49ED5
:041292009024BDF0F7
:011296002235
:101AA7007E247FB81221A99024B9E090E7C1F09075
:101AB70024BAE090E7C2F09024BEE090E7C3F0902C
:101AC70024B7E0600B43A020753AFF1211B28003E0
:101AD700121F9E902452E53AF07A247B527D017FB3
:101AE7002112209C9024527402F0A37480F07A246F
:101AF7007B527D027F2812209CE4902452F0902490
:101B0700BEE0902453F07A247B527D027F28022086
:011B17009C31
:10136B000556E55670020555054D0557B5340DE587
:10137B0055B53308121AA7E4F555F55690E7C8E5AD
:10138B0050F0A3E52CF0A3E539F0E557B40A17901C
:10139B00FC00E0B411097B017AFC7900121C2BE4F0
:1013AB0090FC00F0F557E54DB52B20E5506011246E
:1013BB00FE6008047012122187800D12219980089B
:1013CB00E4FF121F4853A0EFE4F54D30015C754B61
:1013DB000190E7C0E54BF0E5A030E7032009F8905A
:1013EB00F00074AAF0A37411F0A374CCF0A374EE04
:1013FB00F0E490E690F090E6917405F0120E5D909B
:10140B00F00074AAF0A37411F0A374CCF0A374EEE3
:10141B00F0E490E690F090E6917405F0C201E4F5EB
:0B142B004B90E7C0E54BF01221C422FB
:0216FE00D322F5
:0217FE00D322F4
:02222000D322C7
:101B180090E680E030E73A00000090E6207402F09A
:101B2800000000E490E621F000000090E624740232
:101B3800F0000000E490E625F000000090E626742E
:101B480002F0000000E490E627F0000000D20380D5
:101B580016000000E490E620F000000090E62174F2
:0F1B680040F0000000C20390E6BAE0F54CD32233
:10213F0090E740E54CF0E490E68AF090E68B04F0EF
:02214F00D32299
:08220C0090E6BAE0F527D322A9
:1021510090E740E527F0E490E68AF090E68B04F002
:02216100D32287
:02222200D322C5
:02222400D322C3
:02222600D322C1
:10008000E4F56AF56BF56C90E6B9E0120C7200B31A
:10009000B300EBB5029AB602D2BB0324BC0385C2FF
:1000A00003CDC503ECC60421CA0463CB04D7D0003A
:1000B00000058EE490E68AF090E68BF090E6A0E0F2
:1000C00020E1F990E68BE0F56AE4F5B390E601747F
:1000D000CAF0D20100000090E6047480F000000035
:1000E0007402F0000000E4F0020590E490E68AF06B
:1000F00090E68BF090E6A0E020E1F990E68BE0F549
:100100006AD3943F4024E4F56B7440256BF582E498
:1001100034E7F583E0FF7412256BF582E43424F5AF
:1001200083EFF0056BE56BB440DF7F8A7E00122120
:10013000F1902412E0FF7E001221FA902413E07562
:10014000F004A4FFAEF0122203902417E0C394023F
:100150005013902433E090E6C07005744EF0801682
:10016000749CF08011902433E090E6C07005749F79
:10017000F08003749DF0902435E024FF92089024D1
:1001800032E024FF9207902436E024FF920A902464
:1001900040E0754000F541A3E0FEA3E07C002400B0
:1001A000F525EC3EF524902445E09024B6F090240B
:1001B00018E0F536E536700375360190241DE0FE33
:1001C000A3E07C002400F529EC3EF528A3E0FEA383
:1001D000E02400F552EC3EF551902419E0FEA3E036
:1001E0002400F532EC3EF531A3E0FEA3E02400F557
:1001F00054EC3EF55390244DE0FFE4FDFEFBFAF98C
:100200007801120BFFA804A905AA06AB07902423C6
:10021000E0FEA3E07C002400FFEC3EFEE4FDEB2FBB
:10022000FFEA3EFEED39FDEC38FCC004C005C00617
:10023000C00790244EE0FFE4FCFDFEFBFA7901F8D4
:10024000120BFFD003D002D001D000EF2BF54AEE05
:100250003AF549ED39F548EC38F547902421E0FEB0
:10026000A3E07C002400F52FEC3EF52EE4FD7F900A
:10027000122163902413E0FCA3E0FDA3E0FEA3E0C1
:10028000F5468E458D448C43E546F546E545F545F6
:10029000E544F544E4F543020590E4F56B7412255A
:1002A0006BF582E43424F583E0FF7440256BF5821E
:1002B000E434E7F583EFF0056BE56BB440DF000055
:1002C00000E490E68AF000000090E68B7440F002B3
:1002D0000590E490E68AF090E68BF090E6A0E020AE
:1002E000E1F990E6BCE0902452F0E4F56B90E6BEB4
:1002F000E0FFE56BC39F501E7440256BF582E4342C
:10030000E7F583E0FF7453256BF582E43424F5832D
:10031000EFF0056B80D790E6BAE0C313FF90E6BE1E
:10032000E0048059E490E68AF090E68BF090E6A035
:10033000E020E1F990E6BDE0902452F090E6BCE0C8
:10034000902453F0E4F56B90E6BEE0FFE56BC39FAD
:10035000501E7440256BF582E434E7F583E0FF74AA
:1003600054256BF582E43424F583EFF0056B80D7D8
:1003700090E6BAE0C313FF90E6BEE02402FD7A24C3
:100380007B520204D190E7407409F0A37414F0A3E7
:10039000740CF0A37426F0A37407F0A374EEF0A31A
:1003A0007401F0A37403F0A37453F0300305E4A3C5
:1003B000F0800690E74974FFF0000000E490E68AC0
:1003C000F000000090E68B740AF00205907AE77B5B
:1003D000407D047F48122080000000E490E68AF00F
:1003E00000000090E68B7404F0020590E490E68A29
:1003F000F090E68BF090E6A0E020E1F990E68BE04B
:10040000F56AD39401500302059090E741E0FD7F27
:100410004212216390E740E0FD7F4E122163020506
:100420009090E6BCE090256AF07A257B6A7D017F9A
:100430005012209C7A257B6A7D017F5012209C906F
:10044000E6BEE0FD7AE77B407F50122080E490E634
:100450008AF000000090E6BEE090E68BF00000001D
:10046000020590E490E68AF000000090E68BF00030
:10047000000090E6A0E020E1F990E6BCE0D394070C
:100480005003020590E0902452F0E4F56B90E6BE34
:10049000E0FFE56BC39F501E7440256BF582E4348A
:1004A000E7F583E0FF7453256BF582E43424F5838C
:1004B000EFF0056B80D790E6BEE004FD7A247B5216
:1004C0007F5012209C90E6BEE004FD7A247B527F90
:1004D0005012209C020590E490E68AF090E68BF0A2
:1004E00090E6A0E020E1F990E68BE0F56BC29890F1
:1004F000E740E0C394304006E0D39437400790E7EC
:1005000040E0F47076E550707243A01090E740E050
:10051000F4600AE0B4300FE52C64016009D20D7577
:100520005001C20B806A90E740E0C394314061E023
:10053000D39437505BE024D1F52D652C6052C20C6A
:10054000E0B40A03752D6190E740E0B40B03752D0C
:100550006290E740E0B40C03752D6390E740E0B48F
:100560000D03752D6490E740E0B40E03752D659082
:10057000E740E0B40F03752D66800E90E740E0B4CD
:10058000200EE550700A43A0107550028002D3225D
:01059000C3A7
:010591002247
:1020D000C0E0C083C082D2105391EF90E65D7401DE
:0820E000F0D082D083D0E03281
:10210000C0E0C083C0825391EF90E65D7404F0D0CC
:0621100082D083D0E03212
:10211600C0E0C083C0825391EF90E65D7402F0D0B8
:0621260082D083D0E032FC
:101DBE00C0E0C083C08285100C85110D850D828513
:101DCE000C83A37402F085080E85090F850F82859A
:101DDE000E83A37407F05391EF90E65D7410F0D06C
:061DEE0082D083D0E03238
:1020E800C0E0C083C082D2125391EF90E65D7408BD
:0820F800F0D082D083D0E03269
:101D4A00C0E0C083C08290E680E030E72085080CBE
:101D5A0085090D850D82850C83A37402F085100E0A
:101D6A0085110F850F82850E83A37407F05391EFB7
:0D1D7A0090E65D7420F0D082D083D0E0327E
:012228003283
:012229003282
:01222A003281
:01222B003280
:101E9000C0E0C083C08290E65EE054FBF00000002A
:101EA00090E68F7440F00000005391EF90E65FE001
:101EB0004404F090E65EE04404F0D082D083D0E0A9
:011EC00032EF
:10129700C0E0C0F0C083C082C0D075D000C000C01D
:0D12A70001C002C003C004C005C006C0079E
:1012B40075580075590090E65EE054F7F090E6A189
:1012C400E020E1F990E780E0FF1460161460262422
:1012D400D0603A2434604D14605414705675230061
:1012E400805190E782E0F53A90E781E0F54290245E
:1012F400B7E4F0803E90E782E0902410F090E7811C
:10130400E0902411F09024B77401F0802690E781D6
:10131400E070051219C3801B90E781E0B4FF14123A
:1013240021C4800F90E781E024FF92098005752392
:1013340000D20400000090E68DE4F05391EF90E6B3
:0C1344005FE04408F090E65EE04408F032
:10135000D007D006D005D004D003D002D001D000F1
:0B136000D0D0D082D083D0F0D0E0329B
:01222C00327F
:01222D00327E
:101D0B00C0E0C083C08290E65EE054BFF0000000EC
:101D1B0090E6987402F000000090E699E4F0000061
:101D2B000090F800F0A3F05391EF90E65FE0444091
:0F1D3B00F090E65EE04440F0D082D083D0E032FA
:0F1B7700C0E0C083C082C0D075D000C004C006DB
:101B860090E65EE0547FF090E6A6E020E1F990E66C
:101B96009CE0FE90E69DE07C002400F559EC3EF5C5
:101BA6005800000090E69CE4F090E69DF05391EF1B
:0E1BB60090E65FE04480F090E65EE04480F050
:0D1BC400D006D004D0D0D082D083D0E03243
:01222E00327D
:01222F00327C
:01223000327B
:01223100327A
:012232003279
:012233003278
:012234003277
:012235003276
:012236003275
:012237003274
:012238003273
:012239003272
:01223A003271
:01223B003270
:01223C00326F
:01223D00326E
:01223E00326D
:01223F00326C
:01224000326B
:01224100326A
:012242003269
:012243003268
:012244003267
:012245003266
:012246003265
:012247003264
:0618AB008F6D8C6E8D6F45
:1018B100536D0753B0F7122065E4F570C3740295B8
:1018C10070FFE56DA807088002C313D8FC30E0055E
:1018D10043800280035380FD1220651220625380F1
:1018E100FE1220650570E570C3940340CFE4F570E6
:1018F100C374099570FFE56FAE6EA807088005CE29
:10190100C313CE13D8F930E005438002800353801E
:10191100FD1220651220625380FE1220650570E5DC
:1019210070C3940A40CA43B00812206553B0F77FD0
:061931000A7E000220699D
:0921F100AD07AC06E4FF0218ABD7
:0921FA00AD07AC067F040218AB2E
:09220300AD07AC067F010218AB27
:10216300902452EDF0EFC313FF7A247B527D0102DA
:02217300209CAE
:072062004380017F0A7E00AC
:10206900EF7803C333CE33CED8F9FFEF4E6007EFD5
:072079001F70F81E80F52224
:0D21B700D282C283D287C284D286D2852212
:101CC500C2827F017E00122069D284D2867F017E86
:101CD50000122069C2857F017E00122069D283D25D
:101CE500877F017E00122069C2847F017E00122059
:101CF50069D2827F017E00122069C2837F017E0046
:061D0500122069D28522C4
:10201700C284C2867F037E00122069C283C2877F83
:10202700037E00122069C284D2867F037E001220BD
:0620370069C283D287227A
:10217500E4FDFC121CC50DBD00010CBC0AF5BDC873
:01218500F267
:012186002236
:1014F90085463F85453E85443D85433CE52F452E40
:10150900700AC2B17F32FE122069D2B1300705C21A
:10151900B043A0403008030215AA752301E47FE80F
:101529007E03FDFCAB3FAA3EA93DA83CC3120C4E6D
:101539004061E5236401705B7FDD7E031217B812F9
:101549001AA7E53F2418F53FE53E34FCF53EE53D95
:1015590034FFF53DE53C34FFF53CE4FFFEFDE53C99
:10156900FC7818120C5F90E7C4EFF0E4FFFEE53D4C
:10157900FDE4FC7810120C5FA3EFF0E4FFE53EFEFA
:10158900E4FDFC7808120C5FA3EFF0E53FFFA3EF41
:10159900F0808AE523B40112AE3EAF3F1217B8803E
:1015A90009752301E523640160FA300705D2B053B8
:0315B900A0BF22AE
:101678008F728E718D708C6FE4FFFEFDFCAB72AAC9
:1016880071A970A86FD3120C4E4057000000E4FFF8
:10169800FEFDE56FFC7818120C5F90E6CEEFF000C7
:1016A8000000E4FFFEE570FDE4FC7810120C5F908A
:1016B800E6CFEFF0000000E4FFE571FEE4FDFC7802
:1016C80008120C5F90E6D0EFF0000000E572FF9082
:1016D800E6D1EFF000000075BB04000000E5BB3068
:0316E800E7FB22FB
:081D87008C6F8D70AB07AA06FA
:101D8F00E4FDFCC3ED9570EC956F5022EA90E6D020
:101D9F00F0000000EB90E6D1F000000075BB0500ED
:0E1DAF000000E5BB30E7FB0DBD00010C80D548
:011DBD002203
:101FC700AD07AC06000000ED25E0EC3390E6D0F05D
:101FD700000000ED25E090E6D1F000000075BB049D
:091FE700000000E5BB30E7FB221D
:101C7C00E47FD2FEFDFCAB46AA45A944A843D3128F
:101C8C000C4E4026E546242EF546E54534FFF54539
:101C9C00E54434FFF544E54334FFF5431214F9E50C
:101CAC002F452E7011122175800CE52F452E7003D7
:091CBC001221751214F90220171F
:100E5D00C20453A0F043A0047FD07E071220695333
:100E6D00A0F043A00C7FD07E0712206953A0F04361
:100E7D00A0087FD07E071220697FAE1221D1902469
:100E8D00B6E0B40106200503121A35754B0290E742
:100E9D00C0E54BF0121C7C754B0390E7C0E54BF0A1
:100EAD00300403020F96E4F56CF56DC3E56D9529DD
:100EBD00E56C9528501BE4F56EE56EC3953650072D
:100ECD00121CC5056E80F2056DE56D70DE056C803A
:100EDD00DAD3E5419400E5409400400BAD41AC40C0
:100EED00AF32AE31121D87D3E5259400E524940071
:100EFD004007AF25AE24121FC7E4F56AF56BC3E5B5
:100F0D006B9554E56A9553502C121F73E4F56CF5EF
:100F1D006DC3E56D95367480F8656C98500D121C97
:100F2D00C5056DE56D70EA056C80E6056BE56B70CA
:100F3D00CD056A80C9E4F56CF56DC3E56D9552E597
:100F4D006C9551501BE4F56EE56EC3953650071246
:100F5D001CC5056E80F2056DE56D70DE056C80DAE1
:100F6D00D282D283D287D284D286D285AF4AAE497D
:100F7D00AD48AC471216789024B6E0B401062005B2
:090F8D00031219C37FAF1221D138
:010F96002238
:101F7300000000E53225E0E5313390E6D0F00000C3
:101F830000E53225E090E6D1F000000075BB0400C7
:0B1F93000000E5BB20E7033004F8224B
:101BD1000530E530B40803E4F530E53070047F08E2
:101BE100803DE530B401047F0A8034E530B402045D
:101BF1007F02802BE530B403047F038022E530B4FB
:101C010004047F018019E530B405047F058010E5E7
:101C110030B406047F048007E530B4070C7F0C1252
:0A1C21001F487F2D7E00122069226B
:10218700C202E550600B121BD10538E53870020515
:022197003722ED
:10219900E550600B0538E53870020537121BD1226E
:0D21C40053A0F07526FF90E7CBE526F02232
:1019C30053A0F043A0097F287E0A12206953A0F098
:1019D30043A0017F287E0A12206953A0F043A0038D
:1019E3007F287E0A12206953A0F043A0027F287E3D
:1019F3000A12206953A0F043A0067F287E0A122012
:101A03006953A0F043A0047F287E0A12206953A0E3
:101A1300F043A00C7F287E0A12206953A0F043A054
:101A2300087F287E0A122069E4F52690E7CBE52695
:021A3300F0229F
:101A350053A0F043A0087FC47E0912206953A0F08B
:101A450043A00C7FC47E0912206953A0F043A00473
:101A55007FC47E0912206953A0F043A0067FC47E8F
:101A65000912206953A0F043A0027FC47E09122009
:101A75006953A0F043A0037FC47E0912206953A0D7
:101A8500F043A0017FC47E0912206953A0F043A052
:101A9500097FC47E0912206975260190E7CBE526EA
:021AA500F0222D
:08221400E4F51BD2E9D2AF2270
:101DF40090E678E020E6F9C2E990E678E04480F0E5
:101E0400EF25E090E679F090E678E030E0F990E6AE
:101E140078E04440F090E678E020E6F990E678E057
:061E240030E1D6D2E922F4
:101E5E00A90790E678E020E6F9E51B702390E67876
:101E6E00E04480F0E925E090E679F08D16AF03A905
:101E7E00077517018A188919E4F51A751B01D32203
:021E8E00C3226D
:101E2A00A90790E678E020E6F9E51B702590E678A8
:101E3A00E04480F0E925E0440190E679F08D16AFA0
:101E4A0003A9077517018A188919E4F51A751B037E
:041E5A00D322C322AA
:03004B000210AAF6
:1010AA00C0E0C083C082C085C084C086758600C087
:1010BA00D075D000C000C001C002C003C006C0077E
:1010CA0090E678E030E206751B0602119490E67805
:1010DA00E020E10CE51B64026006751B070211940F
:1010EA00E51B24FE605F14603624FE70030211853E
:1010FA0024FC700302119124086003021194AB17B7
:10110A00AA18A919AF1A051A8F82758300120B68DB
:10111A0090E679F0E51A65167070751B05806B907C
:10112A00E679E0AB17AA18A919AE1A8E8275830060
:10113A00120B95751B02E5166401704E90E678E075
:10114A004420F08045E51624FEB51A0790E678E0BB
:10115A004420F0E51614B51A0A90E678E04440F007
:10116A00751B0090E679E0AB17AA18A919AE1A8E7A
:10117A0082758300120B95051A800F90E678E04479
:10118A0040F0751B008003751B005391DFD007D018
:10119A0006D003D002D001D000D0D0D086D084D0DF
:0811AA0085D082D083D0E03231
:10208000121E2AE51B24FA600E146006240770F362
:0C209000D322E4F51BD322E4F51BD3227D
:10209C00121E5EE51B24FA600E146006240770F312
:0C20AC00D322E4F51BD322E4F51BD32261
:03000000021937AB
:0C193700787FE4F6D8FD75817202197EFD
:100B6800BB010CE58229F582E5833AF583E0225042
:100B780006E92582F8E622BBFE06E92582F8E2228C
:0D0B8800E58229F582E5833AF583E49322A6
:100B9500F8BB010DE58229F582E5833AF583E8F096
:100BA500225006E92582C8F622BBFE05E92582C842
:020BB500F2222A
:100BB700EF8DF0A4A8F0CF8CF0A428CE8DF0A42E52
:020BC700FE220C
:100BC900C2D5EC30E709B2D5E4C39DFDE49CFCEE47
:100BD90030E715B2D5E4C39FFFE49EFE120C98C31B
:100BE900E49DFDE49CFC8003120C9830D507C3E416
:060BF9009FFFE49EFE22B6
:100BFF00E88FF0A4CC8BF0A42CFCE98EF0A42CFC95
:100C0F008AF0EDA42CFCEA8EF0A4CDA8F08BF0A412
:100C1F002DCC3825F0FDE98FF0A42CCD35F0FCEB71
:100C2F008EF0A4FEA9F0EB8FF0A4CFC5F02ECD3936
:0F0C3F00FEE43CFCEAA42DCE35F0FDE43CFC22A3
:100C4E00EB9FF5F0EA9E42F0E99D42F0E89C45F0FC
:010C5E002273
:100C5F00E8600FECC313FCED13FDEE13FEEF13FF73
:030C6F00D8F12297
:100C7200D083D082F8E4937012740193700DA3A311
:100C820093F8740193F5828883E473740293686025
:060C9200EFA3A3A380DF25
:101943000209AEE493A3F8E493A34003F68001F203
:1019530008DFF48029E493A3F85407240CC8C333A5
:10196300C4540F4420C8834004F456800146F6DF74
:10197300E4800B0102040810204080900CEDE47E0B
:10198300019360BCA3FF543F30E509541FFEE49369
:10199300A360010ECF54C025E060A840B8E493A330
:1019A300FAE493A3F8E493A3C8C582C8CAC583CA5B
:1019B300F0A3C8C582C8CAC583CADFE9DEE780BE13
:010E5C000095
:100C9800BC000BBE0029EF8DF084FFADF022E4CC40
:100CA800F875F008EF2FFFEE33FEEC33FCEE9DEC09
:100CB800984005FCEE9DFE0FD5F0E9E4CEFD22ED4F
:100CC800F8F5F0EE8420D21CFEADF075F008EF2F99
:100CD800FFED33FD4007985006D5F0F222C398FD8A
:050CE8000FD5F0EA2227
:00000001FF
